:020000040000FA
:020000000428D2
:08000800FF30A200FF30A3004D
:100010008B01B42122101922A210182222111722BA
:10002000FF301A22A501A601A701A801A901AA0172
:10003000AB01AC01AD01AE01AF01B001B201B30142
:10004000FF30B400B501C430E12120168721A01192
:100050008C21A01491217021201D2F2830283128B7
:100060002B288101A01091217021201D38283A28C9
:10007000392834280108B10081013108103C0318E7
:1000800026290130B200A501B301A901AA01AB01E3
:10009000AC01AD01AE01AF01B001FF30B400B5015C
:1000A0003308013C031D5528E6282608A8007021C6
:1000B000201D5B285C2860283308013C031D612853
:1000C0006A280108A6002608C83C031869280130E0
:1000D000B300572881013308013C0319DE282608A4
:1000E0003502031875282608B500340826020318BF
:1000F0007B282608B4002808023EB60026083602EF
:10010000031895283008B8002F08B9002E08BA0047
:100110002D08BB00013096213808B0003908AF0027
:100120003A08AE003B08AD00A7283008B8002F08F9
:10013000B9002E08BA002D08BB00003096213808FF
:10014000B0003908AF003A08AE003B08AD00250802
:10015000A7007021201DAD28AF28AE28A9280108CE
:10016000A50081012708023EB700250837020318C1
:10017000CC282C08B8002B08B9002A08BA00290896
:10018000BB00013096213808AC003908AB003A08B2
:10019000AA003B08A900DE282C08B8002B08B900EB
:1001A0002A08BA002908BB00003096213808AC00A4
:1001B0003908AB003A08AA003B08A900B20A320885
:1001C0001F3C0318E5280130B30050283308013CD8
:1001D000031D2629A014912132081B3C031D26294A
:1001E0004E21A01DF528A014F628A0106121A01E04
:1001F000FA280329FB28A01C0329A0118C217F21A8
:100200000130222226293B21201E082920150929F8
:1002100020116121A01E0D2916290E29201D162945
:10022000A0158C217F210130222226292821A01E01
:100230001B29A0151C29A0116121A01E20292129FC
:100240002629A01D26297F2101302222292827299D
:10025000A0122F08483C031D3A293008023C031D18
:100260003A292E08153C031D3A292D08883C031D08
:100270003A29A016080020122F08413C031D4D29E1
:100280003008023C031D4D292E08943C031D4D29C6
:100290002D080A3C031D4D2920160800A0112F0827
:1002A0004A3C031D60293008023C031D60292E08CA
:1002B000553C031D60292D08953C031D6029A015A0
:1002C0000800B6010330B700861A6729B60AB70BD3
:1002D0006429A0120230360203186F29A016080004
:1002E000B7010330B80086197629B70AB80B73290D
:1002F00020110230370203187E2920150800201231
:100300008721013029220130302220168729A410AC
:10031000201E8B29A414122A2410A01D9029241415
:10032000132A2411A01C95292415112ABC0003109E
:10033000BB0D0310BA0D0310B90D0310B80D8030BA
:100340003B02031CA429BA0A80303A02031CA929E3
:10035000B90A80303902031CAE29B80A3C08003CB7
:100360000318B329BB0A08008B012030DB21BD2113
:10037000803098001030980408001930CC21A01467
:10038000A01CC729D22127080438DB21CB29D22180
:100390002708FB39DB210800A500B7019930B80018
:1003A0002508E729A9019830AA00FC212B08A800FC
:1003B0002808A7000800A500B7019830B800250854
:1003C000E729B600B7018130B8003608E729B9003F
:1003D000831FEC292015ED292011371CF1298317E3
:1003E000F22983133808840039088000201DFA2977
:1003F0008317FB2983130800AB00831F012A2015F4
:10040000022A2011291C062A8317072A83132A0887
:1004100084000008AB00201D0F2A8317102A8313C5
:100420000800142A142A142A2408850008001F2A08
:100430001F2A1F2AA3001C2A23086600080022087E
:1004400065000800B6003608B700FA30B800C830BA
:10045000372AB6003608B7006430B8001430372A9F
:10046000B6003608B7006430B8000530372AB90046
:10047000FF30BA003808BC003708BB0017303A0715
:1004800003183F2ABB0B3E2ABC0B3C2AB90B3A2A65
:02049000080062
:02400E00903FE1
:00000001FF
